:020000040000FA
:0400000004EF00F019
:08000800C20E4CEC00F07BEC91
:1000100000F07AEC00F0FF0E926E936A946A810E03
:10002000046E24EC00F00550026E0650036E025080
:10003000030BFF0A76EC00F00350FF0A78EC00F0A7
:100040000FEF00F022EF00F0066EC2B02CEF00F0D0
:10005000C280010E50EC00F004503EEC00F03CEC8D
:1000600000F038EC00F0C450056EC350066E12006C
:10007000C2B438EF00F01200C2841200076E0750BD
:10008000C26E0750015CD8B449EF00F0010E58EC85
:1000900000F00750016E1200026E0250C16E120095
:1000A000076E0750096E640E0A6E0A0E60EF00F0CC
:1000B000086E0850096E640E0A6E010E60EF00F0C3
:1000C0000B6EFF0E0C6E0A500E6E09500D6EEF0E89
:1000D0000C24D8B068EF00F00D2E67EF00F00E2E64
:1000E00065EF00F00B2E63EF00F012008B6E120034
:0800F0008A6E120012001200DA
:0200000400F00A
:020000040030CA
:0E00000000260E0E00008000F0C00FE00F4042
:00000001FF
